:020000040000FA
:02000000B2D17B
:08000800FACF0BF0EACF0DF076
:10001000E9CF0EF08EED00F0126ED8CF13F0E0CFE6
:1000200011F0FACF0CF0F950D86AEACF0FF0E9CF0F
:1000300010F0F2B409D09EA802D09DB8ADD09EAA0F
:1000400002D09DBA70D0FF008A6A896AFF0E926E54
:10005000896E402A400E406402D0010E406E446A10
:1000600040504160448442604482436044808B50ED
:10007000F80B441009B0070A8B6E90EC01F0F950B0
:100080001850F92638D030D028D020D018D010D031
:1000900008D0301C926E186A800E8A6E39EC01F01E
:1000A00030D02F1C926E0E0E186E400E8A6E29D024
:1000B0002E1C926E0C0E186E200E8A6E22D02D1CF5
:1000C000926E0A0E186E100E8A6E1BD02C1C926E49
:1000D000080E186E080E8A6E14D02B1C926E060E37
:1000E000186E040E8A6E0DD02A1C926E040E186EC5
:1000F000020E8A6E06D0291C926E020E186E010E38
:100100008A6EF29411C0E0FF125013C0D8FF10C0E5
:10011000E9FF0FC0EAFF0CC0FAFF10000600F9501B
:100120009EB266D0FF009E9AABA205D0AB98AE50AF
:10013000AE50AE50AB88ABA402D0AE50E3D7D624BD
:10014000626E5EB4DFD75EB005D0AE50CC0ADAE1A5
:100150005E80D8D75EB207D0AE50F00A01E0D2D7A9
:100160005E82606ACFD701EE00F06050AECFEBFF49
:10017000602A100E6062C6D75E84606A5E905E92EE
:10018000F29E010EFC6E360EFD6E050EFE6E000E2A
:10019000FF6EF950F28E10005EB60DD001EE10F039
:1001A0006350EB50ACA2FED7AD6E632A1B0E6362A8
:1001B000A9D75E86A7D75E96636AAC9AF29E61B0B5
:1001C00007D05E8EFF0E156E166E176E5E8A05D016
:1001D000D6CF01F062C000F05E9E010EFC6EC40E30
:1001E000FD6E040EFE6E000EFF6EF28EF9501000D2
:1001F0009E92377037B036D03866380639EC0FF03B
:10020000E86620D059A41ED0565002620CD055503A
:10021000036209D00830010B356E010E0814351841
:1002200002E1599E0FD0565004620CD05550056221
:1002300009D00830E830010B356E010E081435186E
:1002400001E1598E5D4E07D0020E5D620BD08250E7
:10025000300B5C6E07D0030E5D6E8250300B5C621B
:1002600001D05B6E0EC0E9FF0DC0EAFF0BC0FAFFC4
:1002700011003D6611D019C029F01AC02AF01BC028
:100280002BF01CC02CF01DC02DF01EC02EF01FC086
:100290002FF020C030F012003C2E08D03BC03CF0C4
:1002A0003F2E04D03DC03FF03E2C3E6E3E503C5CA5
:1002B000D8B0E1D721C029F022C02AF023C02BF00A
:1002C00024C02CF025C02DF026C02EF027C02FF022
:1002D00028C030F0120019C021F01AC022F01BC053
:1002E00023F01CC024F01DC025F01EC026F01FC046
:1002F00027F020C028F03BC03EF03BC03CF03DC0A2
:100300003FF050B0120045C048F046C049F047C029
:100310004AF04DC04CF04DC04EF04BC04FF01200B3
:100320004B6608D0506A45C041F046C042F047C015
:1003300043F012004E2E0CD04DC04EF04F2E08D080
:100340004BC04FF04C6602D0506AEDD750804C2E17
:100350004C504E5CD8B0E7D748C041F049C042F09D
:100360004AC043F01200D3507009D36E9B8C00EE4C
:1003700000F0EE50002600B0012AEAA0FAD700EE05
:1003800000F0006602D0450E006E016602D0300E0D
:10039000016E1EEC0FF0D4EC10F00A50AA0A0EE029
:1003A0001EEC0FF00C0E026E0B0E046EF90E076EB3
:1003B000050E086E036A056A066A096AC26A0F0EAC
:1003C000C16E070EB46EFF0E926E896E936AF00EC8
:1003D000946E8A6A8B6A010E3D6E100E3B6E050E9E
:1003E0004B6E400E4D6E0C0E566E556A546A536A33
:1003F0000880300E5B6E050E5D6E616AC10ED56EB3
:10040000D66ACA6ACC6A4B0ECA6E07C0CBFFCA84D2
:10041000080EB86E460EAF6E100EB06E040EAC6EC7
:10042000900EAB6EF26A9D6AA06A9E6AF06AC00E78
:10043000F16E020E9F6ED08E9D829F9A9F989D882E
:100440009D8AE00EF26E82BA20D082B815D0080ED6
:100450001F6E0C0E026E046E036A056A066AF90EC0
:10046000076E086A096A0A6AC8EC10F005EC18F011
:10047000300E5B62FDD7FF00800E1F6E0980C6EC58
:1004800010F005EC18F082AAFCD7FF0E196E1A6E58
:100490001B6E1C6E1D6E1E6E1F6E206E6BEC01F0CF
:1004A000640ECDEC0EF0400E456E466E476EFA0EB1
:1004B000CDEC0EF0FA0ECDEC0EF0F3EC0EF0640E77
:1004C000CDEC0EF016C017F015C016F014C015F0E4
:1004D000DCEC0EF000503F0B146E5EBA09D01562D2
:1004E00001D0F6D7166201D0F3D7176201D0F0D74A
:1004F0005E9A0150070B0109316EDCEC0EF00138F9
:100500001F0B0709396E5EBC09D001500024D624A8
:100510000F0B326E0C0E326042EF1FF0F3EC0EF058
:1005200059BE24EF06F0F950070EFA6E1450040D70
:10053000F35080EF03F05E8C9D9801EE00F0EECF5B
:1005400032F0EECF33F006EC03F0616E646EEECF66
:1005500032F0EECF33F006EC03F0656E64263F0E0A
:10056000656052D0EECF32F0EECF33F006EC03F000
:10057000666E6426EECF32F0EECF33F006EC03F079
:10058000676E6426EECF32F0EECF33F006EC03F068
:10059000686E6426EECF32F0EECF33F006EC03F057
:1005A000696E6426EECF32F0EECF33F006EC03F046
:1005B0006A6E6426EECF32F0EECF33F006EC03F035
:1005C0005E94641821E165C014F066C039F067C01C
:1005D00031F068C001F069C000F0599E6ABE598EC2
:1005E000F3EC0EF061B007D05E8EFF0E156E166E46
:1005F000176E5E8A67D761A006D0D6CF01F062C0C1
:1006000000F05E9E5FD7FF005E945CD73230010B36
:1006100032B6020932BA040932BE080933B21009EF
:0E06200033B6200933BA400933BE80091200F8
:10070000F92603EF04F034EF04F08CEF04F0E0EF8F
:1007100004F00BEF05F01FEF05F03DEF05F058EF8B
:1007200005F069EF05F096EF05F0AEEF05F0C7EFC5
:1007300005F004EF06F024EF06F02DEF06F046EF8B
:1007400006F06DEF06F084EF06F09CEF06F0BAEFCE
:1007500006F077EF07F044EF08F083EF08F0BAEF08
:1007600008F003EF09F0E5EF09F043EF0BF069EF54
:100770000BF0D5EF0BF04DEF0CF074EF0CF096EFA3
:100780000CF0B2EF0CF0E1EF0CF014EF0DF044EFD1
:100790000DF060EF0DF092EF0DF0C2EF0DF0DBEF1A
:1007A0000DF01CEF0EF04FEF0EF06BEF0EF09EEF22
:1007B0000EF062EF02F062EF02F062EF02F062EF21
:1007C00002F062EF02F062EF02F062EF02F062EF1D
:1007D00002F062EF02F062EF02F062EF02F062EF0D
:1007E00002F062EF02F062EF02F062EF02F062EFFD
:1007F00002F062EF02F062EF02F062EF02F062EFED
:1008000002F062EF02F001503F0B1F09316EDCEC89
:100810000EF001501F0B0709396E0150070B4B6E8C
:10082000030B3D6E6BEC01F0DCEC0EF000C019F038
:1008300001C01AF0DCEC0EF000C01BF001C01CF08F
:10084000DCEC0EF000C01DF001C01EF0DCEC0EF080
:1008500000C01FF001C020F024EC0FF03950CDECA7
:100860000EF0312EDFD72ED6090E4B6E030E3D6EE5
:100870006BEC01F0FF0E196E1A6E1B6E1C6E1D6E76
:100880001E6E1F6E206E24EC0FF0C80ECDEC0EF025
:10089000E86A28EC0FF0DCEC0EF001500F0B0109B8
:1008A000396E0150030B3D6E00EE19F0DCEC0EF0DA
:1008B000070E0014E926DCEC0EF0070E0114336E6F
:1008C000FE0E346E3352D8B404D034463450332E36
:1008D000FCD76BEC01F0EFCF34F0EF163450EF6241
:1008E00004D0002AD8B0012ADFD73950CDEC0EF061
:1008F0001966DAD71A66D8D71B66D6D71C66D4D73E
:100900001D66D2D71E66D0D71F66CED72066CCD73D
:10091000C80ECDEC0EF0D6D5090E4B6E030E3D6E13
:100920006BEC01F0640ECDEC0EF0DCEC0EF001503F
:100930000F0B0109396E0150030B3D6E00EE19F0EB
:10094000DCEC0EF0070E0014E926DCEC0EF0070ECE
:100950000114336E010E346E3352D8B404D03446D1
:100960003450332EFCD76BEC01F0EFCF34F0EF12A4
:100970003450EF6204D0002AD8B0012ADFD73950B2
:10098000CDEC0EF0FF0E1918D9E1FF0E1A18D6E1C2
:10099000FF0E1B18D3E1FF0E1C18D0E1FF0E1D182F
:1009A000CDE1FF0E1E18CAE1FF0E1F18C7E1FF0EB2
:1009B0002018C4E124EC0FF0C80ECDEC0EF082D567
:1009C000F3EC0EF0DCEC0EF001503F0B0F09316E32
:1009D000DCEC0EF001380F0B0709396E00EE19F050
:1009E000DCEC0EF0070E0014E926DCEC0EF0070E2E
:1009F0000114336E010E346E3352D8B404D0344631
:100A00003450332EFCD7EF6E3950CDEC0EF0EF6A38
:100A1000312EE4D757D5100E336EF3EC0EF0D8908C
:100A20003930CDEC0EF0FFEC0EF03950CDEC0EF07D
:100A3000380E3318D8A4F1D7312EEDD743D5015055
:100A4000030B4B6E3D6E3950CDEC0EF06BEC01F0AC
:100A5000FF0E196E1A6E1B6E1C6E1D6E1E6E1F6EC3
:100A6000206E24EC0FF03950CDEC0EF06BEC01F061
:100A7000F3EC0EF0312EE7D725D5F3EC0EF0030E94
:100A80003116070E336EEA6A190EE96E010E346EE6
:100A900001D034463450EF6E080ECDEC0EF0EF6A04
:100AA00034AEF7D7E92A332EF1D7312EEAD70AD55B
:100AB000050E346E600E336E6BEC01F0FFEC0EF041
:100AC0003950CDEC0EF0342E5CEF05F0312EF0D71E
:100AD000F9D4DCEC0EF001503F0B0F09396E0150D8
:100AE000030B3D6E010B4B6EDCEC0EF0070E011498
:100AF000F66E300EF76E08006BEC01F0F550196ED3
:100B00001A6E1B6E1C6E1D6E1E6E1F6E206E030E07
:100B1000F66402D0E86A02D0F650010F28EC0FF01C
:100B20003950CDEC0EF0312EDFD7CCD4090E4B6E00
:100B3000030E3D6E6BEC01F0F3EC0EF03950CDEC92
:100B40000EF0336A6BEC01F024EC0FF0FFEC0EF0CA
:100B50003950CDEC0EF0312EE9D7B4D4F3EC0EF0D1
:100B6000010E346E01D034466BEC01F03450196E36
:100B70001A6E1B6E1C6E1D6E1E6E1F6E206E39501F
:100B8000CDEC0EF034AEEFD7312EEAD79BD4060E63
:100B90004B6EF3EC0EF0800E1F6E3950CDEC0EF064
:100BA000F3EC0EF0800E206E3950CDEC0EF0F3EC2D
:100BB0000EF0800E1C6E3950CDEC0EF0F3EC0EF002
:100BC000800E1E6E3950CDEC0EF0F3EC0EF0800E60
:100BD0001D6E3950CDEC0EF0312ED9D7F3EC0EF05E
:100BE000040E28EC0FF0800E1F6E206E1C6E1E6E21
:100BF0001D6E640ECDEC0EF06BEC01F0F3EC0EF01C
:100C00003C0ECDEC0EF05ED4F3EC0EF00150030B75
:100C10003D6E010B4B6E3950CDEC0EF03950CDECE2
:100C20000EF06BEC01F024EC0FF0380E336E6BEC31
:100C300001F0FFEC0EF03950CDEC0EF0600E336297
:100C4000F6D7312EE1D73ED4F3EC0EF0C80ECDEC42
:100C50000EF05EAC42EF1FF035D4F3EC0EF0010E57
:100C6000346E01D034466BEC01F0345019121A1274
:100C70001B121C121D121E121F1220123950CDEC15
:100C80000EF034AEEFD7312EE8D71CD4060E4B6EE3
:100C9000DCEC0EF0030E01143D6EF66E300EF76EB6
:100CA00009006BEC01F0F550196E1A6E1B6E1C6E8C
:100CB0001D6E1E6E1F6E206E24EC0FF0C80ECDEC64
:100CC0000EF0C80ECDEC0EF06BEC01F0F3EC0EF074
:100CD000320ECDEC0EF062EF02F0F3EC0EF0060EE9
:100CE0004B6EDCEC0EF0030E01143D6E6BEC01F06C
:100CF000336AFFEC0EF024EC0FF03950CDEC0EF01F
:100D0000312EF9D762EF02F0F3EC0EF0060E4B6EC7
:100D1000DCEC0EF0030E01143D6E6BEC01F0080EDE
:100D2000336EFFEC0EF024EC0FF03950CDEC0EF0EA
:100D3000312EF9D762EF02F0060E4B6EDCEC0EF0AE
:100D4000030E01143D6EF3EC0EF06BEC01F0336A10
:100D5000FFEC0EF03950CDEC0EF06BEC01F0080E0C
:100D6000336EFFEC0EF03950CDEC0EF0312EEBD798
:100D700062EF02F03150030B316E3D6A4B6AF3ECC7
:100D80000EF0800E1F6E3950CDEC0EF03950CDECC8
:100D90000EF0F3EC0EF0400E1F6E200E206E395058
:100DA000CDEC0EF0F3EC0EF0030E196E3950CDECD5
:100DB0000EF0F3EC0EF0600E196E3950CDEC0EF023
:100DC000F3EC0EF0030E1A6E3950CDEC0EF0F3EC8E
:100DD0000EF0100E1C6E100E1E6E3950CDEC0EF083
:100DE000F3EC0EF0020E1C6E020E1D6E3950CDECAF
:100DF0000EF0F3EC0EF0100E206E100E1D6E39503A
:100E0000CDEC0EF0F3EC0EF0800E206E800E1D6E19
:100E10003950CDEC0EF0F3EC0EF0200E1C6E400EAF
:100E20001E6E3950CDEC0EF0F3EC0EF0020E1B6E80
:100E3000010E206E3950CDEC0EF0F3EC0EF0200ECA
:100E40001B6E400E1A6E3950CDEC0EF0F3EC0EF026
:100E5000010E1B6E010E1F6E3950CDEC0EF0F3EC3F
:100E60000EF0400E1B6E200E1A6E3950CDEC0EF0B7
:100E7000F3EC0EF0010E1C6E020E1F6E3950CDEC1D
:100E80000EF0F3EC0EF0400E206E200E1F6E395067
:100E9000CDEC0EF0F3EC0EF0800E1C6E800E1E6E8C
:100EA0003950CDEC0EF0F3EC0EF0400E1C6E200E1F
:100EB0001E6E3950CDEC0EF0F3EC0EF0010E1D6EEF
:100EC000020E1E6E3950CDEC0EF0F3EC0EF0600EFB
:100ED0001D6E3950CDEC0EF0F3EC0EF0010E1E6ECF
:100EE0003950CDEC0EF0312E4AD762EF02F031507E
:100EF000030B316E0150030B3D6E4B6AF3EC0EF0A9
:100F00006BEC01F0800E1F123950CDEC0EF0395011
:100F1000CDEC0EF06BEC01F0400E1F12200E2012F3
:100F20003950CDEC0EF06BEC01F0030E1912395074
:100F3000CDEC0EF06BEC01F0600E19123950CDECD7
:100F40000EF06BEC01F0030E1A123950CDEC0EF0DE
:100F50006BEC01F0100E1C12100E1E123950CDEC6D
:100F60000EF06BEC01F0020E1C12020E1D12395035
:100F7000CDEC0EF06BEC01F0100E2012100E1D12D5
:100F80003950CDEC0EF06BEC01F0800E2012800E8B
:100F90001D123950CDEC0EF06BEC01F0200E1C123E
:100FA000400E1E123950CDEC0EF06BEC01F0020E2B
:100FB0001B12010E20123950CDEC0EF06BEC01F03B
:100FC000200E1B12400E1A123950CDEC0EF06BECB5
:100FD00001F0010E1B12010E1F123950CDEC0EF064
:100FE0006BEC01F0400E1B12200E1A123950CDECA2
:100FF0000EF06BEC01F0010E1C12020E1F123950A4
:10100000CDEC0EF06BEC01F0400E2012200E1F1202
:101010003950CDEC0EF06BEC01F0800E1C12800EFE
:101020001E123950CDEC0EF06BEC01F0400E1C128C
:10103000200E1E123950CDEC0EF06BEC01F0010EBB
:101040001D12020E1E123950CDEC0EF06BEC01F0A9
:10105000600E1D123950CDEC0EF06BEC01F0010E5C
:101060001E123950CDEC0EF024EC0FF0640ECDECD6
:101070000EF06BEC01F0F3EC0EF03950CDEC0EF00D
:10108000312E3CD762EF02F00150030B3D6E4B6AEC
:10109000F3EC0EF06BEC01F0C00E1F12200E2012CC
:1010A0003950CDEC0EF0F3EC0EF06BEC01F0900E3D
:1010B0001D12400E1E123950CDEC0EF0F3EC0EF066
:1010C0006BEC01F0A00E1E12200E1F123950CDEC59
:1010D0000EF0F3EC0EF06BEC01F0C00E1C12400EA3
:1010E00020123950CDEC0EF0F3EC0EF06BEC01F069
:1010F000900E2012200E1C123950CDEC0EF0312E25
:10110000C7D762EF02F0F3EC0EF00C0E1912080EC6
:101110001F123950CDEC0EF0F3EC0EF0040E1C1241
:10112000040E1B12040E20123950CDEC0EF0F3EC1D
:101130000EF0080E1B12080E1C12080E1D1239505C
:10114000CDEC0EF0F3EC0EF0040E1D12040E1E1288
:10115000040E1F123950CDEC0EF0F3EC0EF00C0E15
:101160001A12080E1E123950CDEC0EF0312ECBD7CC
:1011700062EF02F0F3EC0EF0C80E1F12200E2012E8
:101180000C0E19123950CDEC0EF0F3EC0EF0900E5F
:101190001D12400E1E12040E1C12040E1B12040E11
:1011A00020123950CDEC0EF0F3EC0EF0A00E1E1212
:1011B000200E1F12080E1B12080E1C12080E1D1204
:1011C0003950CDEC0EF0F3EC0EF0C00E1C12400EB8
:1011D0002012040E1D12040E1E12040E1F1239508E
:1011E000CDEC0EF0F3EC0EF0900E2012200E1C123F
:1011F0000C0E1A12080E1E123950CDEC0EF0312EC4
:10120000B9D762EF02F00150030B3D6E4B6ADCEC84
:101210000EF001501F0B0709396E030E3116F3EC67
:101220000EF06BEC01F0010E1A123950CDEC0EF0FD
:101230006BEC01F0010E1B123950CDEC0EF06BEC93
:1012400001F0010E1E123950CDEC0EF06BEC01F0E6
:10125000010E1F123950CDEC0EF06BEC01F0020EB6
:101260001A123950CDEC0EF06BEC01F0100E1C127E
:10127000200E1B123950CDEC0EF06BEC01F0400E3D
:101280001B12400E1D123950CDEC0EF06BEC01F02C
:10129000200E1A12200E1D123950CDEC0EF06BEC00
:1012A00001F0100E1E12400E1A123950CDEC0EF045
:1012B0006BEC01F0600E19123950CDEC0EF06BECB6
:1012C00001F0020E1B12020E1C123950CDEC0EF072
:1012D0006BEC01F0010E1C12010E1D123950CDEC09
:1012E0000EF06BEC01F0020E1E12020E1F123950AE
:1012F000CDEC0EF06BEC01F0010E2012020E1D126F
:101300003950CDEC0EF06BEC01F0030E1912395090
:10131000CDEC0EF06BEC01F0100E2012200E1C1222
:101320003950CDEC0EF06BEC01F0400E2012400E67
:101330001C123950CDEC0EF06BEC01F0200E1E1299
:10134000200E1F123950CDEC0EF06BEC01F0100E98
:101350001D12400E1E123950CDEC0EF06BEC01F058
:10136000200E2012400E1F123950CDEC0EF06BEC07
:1013700001F0800E20123950CDEC0EF06BEC01F034
:10138000800E1C123950CDEC0EF06BEC01F0800E8B
:101390001E123950CDEC0EF06BEC01F0800E1D12D8
:1013A0003950CDEC0EF06BEC01F0800E1F1239506D
:1013B000CDEC0EF024EC0FF0640ECDEC0EF06BECE7
:1013C00001F0312E2CD762EF02F0F3EC0EF0800E1C
:1013D0001F6E400E196E3950CDEC0EF0F3EC0EF08E
:1013E000200E206E010E196E3950CDEC0EF0F3EC8C
:1013F0000EF0020E196E400E1F6E3950CDEC0EF03D
:10140000F3EC0EF0200E196E800E1F6E3950CDECED
:101410000EF0F3EC0EF0020E1A6E200E206E395014
:10142000CDEC0EF0F3EC0EF0100E1E6E020E196EE7
:101430003950CDEC0EF0F3EC0EF0020E1D6E200EC6
:10144000196E3950CDEC0EF0F3EC0EF0100E1D6E4F
:10145000020E1A6E3950CDEC0EF0F3EC0EF0800E49
:101460001D6E100E1E6E3950CDEC0EF0F3EC0EF02A
:10147000400E1E6E020E1D6E3950CDEC0EF0F3ECD8
:101480000EF0010E206E100E1D6E3950CDEC0EF0D8
:10149000F3EC0EF0400E1A6E800E1D6E3950CDEC3E
:1014A0000EF0F3EC0EF0010E1F6E400E1E6E395062
:1014B000CDEC0EF0F3EC0EF0200E1A6E010E206E45
:1014C0003950CDEC0EF0F3EC0EF0020E1F6E400E14
:1014D0001A6E3950CDEC0EF0F3EC0EF0210E1F6EAB
:1014E0003950CDEC0EF0F3EC0EF0800E1E6E200E97
:1014F0001A6E3950CDEC0EF0F3EC0EF0200E1E6E8D
:10150000020E1F6E3950CDEC0EF0F3EC0EF0020E11
:101510001E6E200E1F6E3950CDEC0EF0F3EC0EF067
:10152000200E1D6E800E1E6E3950CDEC0EF0F3ECC9
:101530000EF0210E1E6E3950CDEC0EF0F3EC0EF0D5
:10154000400E1D6E020E1E6E3950CDEC0EF0F3EC07
:101550000EF0210E1D6E3950CDEC0EF0F3EC0EF0B6
:10156000400E1C6E010E1E6E3950CDEC0EF0F3ECE9
:101570000EF0800E1C6E400E1D6E3950CDEC0EF03C
:10158000F3EC0EF0400E206E010E1D6E3950CDECC6
:101590000EF0F3EC0EF0410E1C6E3950CDEC0EF057
:1015A000F3EC0EF0400E1B6E800E1C6E3950CDEC2D
:1015B0000EF0F3EC0EF0010E1B6E400E206E395053
:1015C000CDEC0EF0F3EC0EF0200E1B6E010E1C6E37
:1015D0003950CDEC0EF0F3EC0EF0420E1B6E39508C
:1015E000CDEC0EF0F3EC0EF0200E1C6E010E1B6E17
:1015F0003950CDEC0EF0F3EC0EF0800E206E200E84
:101600001B6E3950CDEC0EF0F3EC0EF0100E206E88
:10161000020E1B6E3950CDEC0EF0F3EC0EF0220EE4
:101620001C6E3950CDEC0EF0F3EC0EF0100E1C6E6B
:10163000800E206E3950CDEC0EF0F3EC0EF0010E62
:101640001A6E100E206E3950CDEC0EF0F3EC0EF049
:10165000400E196E020E1C6E3950CDEC0EF0F3ECFC
:101660000EF0010E196E100E1C6E3950CDEC0EF0FE
:10167000F3EC0EF0400E1F6E010E1A6E3950CDECD9
:101680000EF062EF02F0DCEC0EF00150070B4B6E37
:10169000030B3D6E6BEC01F0F3EC0EF0050E346EB7
:1016A0003950CDEC0EF0580E336E6BEC01F0FFECC0
:1016B0000EF0100E335E3950CDEC0EF0342EF5D70F
:1016C00024EC0FF03950CDEC0EF0312EE3D762EF61
:1016D00002F0F3EC0EF0800E1F6E800E1D6E800E79
:1016E0001E6E800E1C6E800E206E3950CDEC0EF0FA
:1016F000F3EC0EF0700E206E600E1E6E3950CDECC5
:101700000EF0F3EC0EF0020E196E010E206E020EBA
:101710001E6E030E1C6E3950CDEC0EF0F3EC0EF085
:10172000200E196E400E1A6E200E1D6E400E1B6E9E
:10173000100E1C6E3950CDEC0EF0F3EC0EF0030ED3
:101740001A6E010E1F6E010E1E6E010E1B6E3950B9
:10175000CDEC0EF0F3EC0EF0100E1E6E200E1A6E95
:10176000400E1D6E200E1B6E400E196E3950CDECD2
:101770000EF0F3EC0EF0030E1D6E020E1F6E020E45
:101780001B6E010E196E3950CDEC0EF0F3EC0EF01D
:10179000100E1D6E600E1F6E600E1C6E3950CDEC6B
:1017A0000EF0312E96D762EF02F0DCEC0EF0015015
:1017B000070B3D6E4B6A6BEC01F0F3EC0EF00C0E78
:1017C000196E3950CDEC0EF03950CDEC0EF06BECBB
:1017D00001F0F3EC0EF0030E1A6E3950CDEC0EF062
:1017E0006BEC01F0F3EC0EF0100E1C6E100E1E6E82
:1017F0003950CDEC0EF06BEC01F0F3EC0EF0020E74
:101800001C6E020E1D6E3950CDEC0EF06BEC01F02B
:10181000F3EC0EF0100E206E100E1D6E3950CDEC54
:101820000EF06BEC01F0F3EC0EF0800E206E800EEB
:101830001D6E3950CDEC0EF03950CDEC0EF06BEC46
:1018400001F0F3EC0EF0100E206E100E1D6E3950EC
:10185000CDEC0EF06BEC01F0F3EC0EF0020E1C6E12
:10186000020E1D6E3950CDEC0EF06BEC01F0F3EC76
:101870000EF0100E1C6E100E1E6E3950CDEC0EF0D8
:101880006BEC01F0F3EC0EF0030E1A6E3950CDEC58
:101890000EF0312E90D762EF02F0F3EC0EF0100E46
:1018A000196E3950CDEC0EF0F3EC0EF0100E1F6EE9
:1018B0003950CDEC0EF0F3EC0EF0100E1A6E3950DC
:1018C000CDEC0EF0F3EC0EF0800E196E3950CDEC2D
:1018D0000EF0F3EC0EF0100E1B6E3950CDEC0EF046
:1018E000312EDBD762EF02F0F3EC0EF04B6A030E01
:1018F00028EC0FF0E86A336EFFEC0EF0800E1F123A
:1019000020121C121E121D123950CDEC0EF039504F
:10191000CDEC0EF01F9E209E1C9E1E9E1D9E3950DB
:10192000CDEC0EF0312EEAD762EF02F0F3EC0EF0C0
:10193000040E326E0F0E336E060E346E800E1F12C2
:1019400020121C121E121D123350CDEC0EF0F3ECBF
:101950000EF03450CDEC0EF0322EF0D7312EE6D70B
:1019600062EF02F0DCEC0EF00150070B3D6E360E1C
:10197000F76E326A00C033F00F0E391633B20ED054
:101980006BEC01F0325030EC1BF03950CDEC0EF026
:10199000322A0B0E3264F2D733B00ED00B0E326EF9
:1019A0006BEC01F0325030EC1BF03950CDEC0EF006
:1019B0003206FF0E3262F4D7326A312EDFD762EF81
:1019C00002F0DCEC0EF00150070B3D6E4B6E030E87
:1019D00028EC0FF0330EF76E326A00C033F00F0EB2
:1019E000391633B20ED06BEC01F0325030EC1BF0F4
:1019F0003950CDEC0EF0322A050E3264F2D733B0F6
:101A00000ED0050E326E6BEC01F0325030EC1BF054
:101A10003950CDEC0EF03206FF0E3262F4D7326A46
:101A2000312EDFD762EF02F0DCEC0EF00150070B35
:101A30003D6E4B6E320EF76E326A00C033F00F0E01
:101A4000391633B20ED06BEC01F0325030EC1BF093
:101A50003950CDEC0EF0322A0B0E3264F2D733B08F
:101A60000ED00B0E326E6BEC01F0325030EC1BF0EE
:101A70003950CDEC0EF03206FF0E3262F4D7326AE6
:101A8000312EDFD762EF02F0DCEC0EF00150070BD5
:101A90003D6E4B6E070E3916370EF76E326A6BECE1
:101AA00001F0325030EC1BF03950CDEC0EF0322A00
:101AB000330E3264F4D7640ECDEC0EF062EF02F018
:101AC000030E3112DCEC0EF00150010B3D6E4B6E3B
:101AD00024EC0FF0390EF76E326A00C033F033B2E7
:101AE0000ED06BEC01F0325030EC1BF03950CDECE5
:101AF0000EF0322A040E3264F2D733B00ED0040E48
:101B0000326E6BEC01F0325030EC1BF03950CDEC02
:101B10000EF03206FF0E3262F4D7326A312EDFD772
:101B200062EF02F0030E3112DCEC0EF00150010BFB
:101B30003D6E4B6E3A0EF76E326A00C033F033B230
:101B40000ED06BEC01F0325030EC1BF03950CDEC84
:101B50000EF0322A040E3264F2D733B00ED0040EE7
:101B6000326E6BEC01F0325030EC1BF03950CDECA2
:101B70000EF03206FF0E3262F4D7326A312EDFD712
:101B800062EF02F0050E4B6E030E3D6E030E311236
:101B90006BEC01F0390EF76E280EF66E33EC1BF08D
:101BA0006BEC01F024EC0FF0640ECDEC0EF0312E56
:101BB000F7D762EF02F0010E3D6E040E3126310EB2
:101BC000F76E09D06BEC01F0680EF66E33EC1BF08B
:101BD000640ECDEC0EF06BEC01F0700EF66E33EC93
:101BE0001BF0140ECDEC0EF06BEC01F0780EF66EDF
:101BF00033EC1BF0140ECDEC0EF06BEC01F0800E0C
:101C0000F66E33EC1BF0640ECDEC0EF06BEC01F0D5
:101C1000780EF66E33EC1BF0140ECDEC0EF06BEC80
:101C200001F0700EF66E33EC1BF0140ECDEC0EF0DE
:101C3000312EC8D762EF02F0030E3112DCEC0EF049
:101C40000150010B3D6E4B6E0B0E28EC0FF03B0E5E
:101C5000F76E326A00C033F033B20ED06BEC01F095
:101C6000325030EC1BF03950CDEC0EF0322A040E1D
:101C70003264F2D733B00ED0040E326E6BEC01F04A
:101C8000325030EC1BF03950CDEC0EF03206FF0E26
:101C90003262F4D7326A312EDFD762EF02F0010EE2
:101CA0003D6E030E31123B0EF76E6BEC01F0280E09
:101CB000F66E33EC1BF03C0ECDEC0EF06BEC01F04D
:101CC000300EF66E33EC1BF0280ECDEC0EF0312EFC
:101CD000ECD762EF02F0030E3112DCEC0EF0015093
:101CE000010B3D6E4B6E0A0E28EC0FF03C0EF76EAA
:101CF000326A00C033F033B20ED06BEC01F03250D8
:101D000030EC1BF03950CDEC0EF0322A040E326468
:101D1000F2D733B00ED0040E326E6BEC01F03250BD
:101D200030EC1BF03950CDEC0EF03206FF0E326273
:101D3000F4D7326A312EDFD762EF02F0030E311290
:101D4000DCEC0EF00150010B3D6E3D0EF76E326A79
:101D500000C033F033B20ED06BEC01F0325030ECF7
:101D60001BF03950CDEC0EF0322A040E3264F2D75B
:101D700033B00ED0090E326E6BEC01F0325030EC05
:101D80001BF03950CDEC0EF03206040E3262F4D75F
:101D9000326A312EDFD762EF02F0386E5BA853EC67
:101DA0000FF05BBA06D0597E5BAAFED7060062EF41
:101DB00002F03866F3D71200016604D0300E5EAE32
:101DC000D624016E006602D0450E006E0134011863
:101DD000E836013A0038E8460118013A010B0036AE
:101DE000001A01361200196A1A6A1B6A1C6A1D6AF7
:101DF0001E6A1F6A206A506AE86A2AD0120033C03D
:101E0000F6FF310EF76E0900F5CF19F00900F5CF96
:101E10001AF00900F5CF1BF00900F5CF1CF00900FE
:101E2000F5CF1DF00900F5CF1EF00900F5CF1FF02A
:101E30000900F5CF20F0080E3326120000EE02F064
:101E4000EE6AE9AEFDD71200DCEC0EF000501F0B7D
:101E500050B01200040DF3CFF6FF3E0EF76E0900EE
:101E6000F5CF45F00900F5CF46F00900F5CF47F072
:101E70001200532A630E5364010C536A5A2A542ADF
:101E80003B0E5464010C546A552A3B0E5564000CF9
:101E9000556A562A0C0E566201D008705664000C22
:101EA000010E566E000C598459904B6A3D6AE86ADF
:101EB00028EC0FF05A6A030E5A6028D0F3EC0EF0AB
:101EC0006BEC01F05BA8F7D7560408EC10F008B0F3
:101ED000278E27C01FF05BBA04D048EC0FF005EC4A
:101EE00010F05BB8F1D7F3EC0EF002EC10F05550A7
:101EF00026EC10F05BBA04D098EC10F005EC10F072
:101F00005BA877D0780E5A64F2D773D05982F3EC7D
:101F10000EF0010E28EC0FF002EC10F0020408ECB9
:101F200010F008B2278E27C01FF05BBA05D0A0ECD6
:101F300010F005EC10F059805BB8F0D7F3EC0EF020
:101F4000010E28EC0FF002EC10F0035026EC10F01C
:101F50005BBA04D0AAEC10F005EC10F05BA804D03A
:101F6000780E5A64F2D745D05982F3EC0EF0020E87
:101F700028EC0FF002EC10F0040408EC10F008B4A8
:101F8000278E27C01FF05BBA04D0B0EC10F005EC30
:101F900010F05BB8F1D7F3EC0EF0020E28EC0FF066
:101FA00002EC10F0055026EC10F05BBA05D0BAEC4C
:101FB00010F005EC10F059805BA804D0780E5A643C
:101FC000F1D717D05982F3EC0EF0030E28EC0FF086
:101FD00002EC10F06DEC10F05BBA05D0C0EC10F024
:101FE00005EC10F059805BA804D0780E5A64F2D743
:101FF00000D002EC10F0599259B0C6EC10F0599094
:10200000599E12005BA8FED712005BAAFED71200F1
:10201000080DF3CFF6FF320EF76E0900F5CF19F079
:102020000900F5CF1AF00900F5CF1BF00900F5CF34
:102030001CF00900F5CF1DF00900F5CF1EF00900D6
:10204000F5CF27F00900F5CF20F012008FEC10F04B
:102050005750080DF3CFF6FF330EF76E0900F5CF9A
:1020600021F00900F5CF22F00900F5CF23F0090097
:10207000F5CF24F00900F5CF25F00900F5CF26F0C3
:102080000900F5CF27F00900F5CF28F05850080DCA
:10209000F3CFF6FF340EF76E0900F5502110196EDC
:1020A0000900F55022101A6E0900F55023101B6E1E
:1020B0000900F55024101C6E0900F55025101D6E06
:1020C0000900F55026101E6E0900F55027101F6EEE
:1020D0000900F5502810206E12000650080DF3CFAD
:1020E000F6FF350EF76E0900F5CFCBFFF5CF07F001
:1020F000196A0900F5CF1AF00900F5CF1BF00900A5
:10210000F5CF1CF00900F5CF1DF00900F5CF1EF04A
:102110000900F5CF1FF00900F5CF20F01200586E2E
:10212000576A0A0E585CD8A01200586E572AF9D781
:10213000536A546A552A3B0E55641200556A1200C0
:10214000022A0C0E026201D0087202641200010E13
:10215000026E1200032A3B0E03641200036A12008F
:10216000042A0C0E046201D0087404641200010EEB
:10217000046E1200052A3B0E05641200056A120067
:10218000062A0E0E06641200066A1200AA0E0A6ED5
:10219000516A090E526E00EE02F0EE50E1EC10F0C2
:1021A000512A522EFAD71200516A090E526E00EED1
:1021B00002F05150F2EC10F0EE6E512A522EF9D787
:1021C0001200A6B2FED7A86E51C0A9FFA69EA69C7B
:1021D000A684F29E550EA76EAA0EA76EA682F28E58
:1021E000A6941200A96EA69EA69CA680A8501200D6
:10300000030CF0FF0FF3FC00FC00230E326EB90E30
:10301000336E090E346E322EFED7332EFCD7342E8B
:04302000FAD71200C9
:103100009C1C1C0C0C0C1C04636363F3F3F3E3F1D1
:10311000632F45C561A3E3600C632B32BAF323919F
:10312000634345C5D751C561632F2B3228A3E3B054
:103130000C4363F3D75105D10003010000010100E6
:103140006063611060110100636363136313030123
:103150006363637373736371636363F3F3F3E3F143
:10316000630300000000C0200042000092500101F3
:103170000020000020A32300000041C141010040C5
:08318000000123320000009061
:1032000000000000800000000000000090000000AE
:10321000000000009200000000000000921000007A
:103220000002000092100000040200009210000052
:103230000C020000921000000C030000921000002D
:103240000C030010921000000C03001292100000FA
:103250000C030012921000100C0300129210009048
:1033000000000000000000001000000000000000AD
:1033100010001000000000009000100000000000ED
:10332000901010000000000090101000000010002D
:10340000000000000000000000000000008000003C
:103410000000000000A000000000000000A200006A
:103420000000000020A200000000000020A3000017
:103430000000000060A300000000000061A3000085
:103440000000004061A30000000000C061A3000074
:10350000F900000000010000F800000008010000C0
:10351000F700080008010000F6000900080100009B
:10352000F500290008010000F4002B00080100004C
:10353000F3002B2008010000F2002B20080100807E
:10354000FA00000004010000FB0000000401040078
:10355000FC00000004010500FD400000040105001E
:10356000FE40000004010501FF4000000441050188
:08357000FF4000008441050149
:10360000000000008000000000000000100000002A
:103610000000000002000000000000000010000098
:103620000002000000000000040000000000000094
:103630000800000000000000000100000000000081
:103640000000001000000000000000020000000068
:1036500000000000000000100000000000000080DA
:10366000080DF3CFF6FF0900F5CF19F00900F5CFEB
:103670001AF00900F5CF1BF00900F5CF1CF0090086
:10368000F5CF1DF00900F5CF1EF00900F5CF1FF0B2
:083690000900F5CF20F0120043
:103700000000000000000000000000000000008039
:103710000000000000000090000000020000009087
:103720000000001200000090000100120000009054
:1037300008010012000000900C010012000000902F
:103740000C030012000000900C0300120010009007
:103750000C030012021000900C03001212100090D3
:103760000C030012921000900C0300129250009073
:103770000C030012925000910C43001292500091E1
:103780000C430012925001910C430012925005918B
:103790000C430012965005910C430012965105916E
:1037A0000C430012D65105910C430012D6510591DD
:1037B0000C430012D75105910C430052D75105918B
:1037C0000C4300D2D75105910C4300D2D75105D1FB
:1037D0000C4300D3D75105D10C4340D3D75105D169
:1037E0000C4341D3D75105D10C4345D3D75105D113
:1037F0000C4345D7D75105D14C4345D7D75105D1B7
:103800004D4345D7D75105D14D4345D7D75145D124
:103810004D4345D7D751C5D14D4345D7D751C5F1B4
:103820004F4345D7D751C5F16F4345D7D751C5F160
:103830006F4745D7D751C5F16F4F45D7D751C5F120
:103840006F6F45D7D751C5F16F6F45D7D751C7F1C6
:103850006F6F45D7D751E7F16F6F45D7D7D1E7F1F4
:103860006F6F45D7D7F1E7F16F6F45D7D7F3E7F122
:103870006F6F45D7F7F3E7F16F6F45D7FFF3E7F1C8
:103880006F6F4DD7FFF3E7F16F6F6DD7FFF3E7F180
:103890006F6F6FD7FFF3E7F16F6F6FF7FFF3E7F12C
:103900009C1018080C041C00901C1C0C08081004C7
:103910009C10140404041C049C1C180808081800BB
:10392000901C1404040C1404030303838383838115
:103A00000C03001292100090004000C0C541050157
:103A1000410145850000C040222E00000080A32007
:083A200000002B2028A3008008
:103B000022020000921090200070000080C023016B
:103B1000800000C061A30000000073A1000000C08D
:103B2000510100120000C09000402B208C41058103
:083B3000000000C061A30000C9
:103C00000C03000000000000000E00000000010096
:103C10000000000004010500000009000801000088
:083C2000000105040000000092
:103D0000410100000000C00000020000921000000D
:103D10000020000000802300000000C041010000DE
:103D200000002320000000800040000080400101CE
:103D30000000000020A300000000418100000040BE
:103D4000000100120000009022020000000080200C
:103E000000000000400000000040000000004000F2
:103E10004040400020000000002000000000200082
:103E2000202020000A000000000A000000000A0014
:103E30000A0A0A00400040004040000000404000E4
:103E400040280000190D4000330D4000400D3300A4
:103E5000400D1900401A0D0040331A0033400D0088
:103E60001A400D000D401A000D4033000D33400084
:103E70000D1A4000000E3A002B003A003A000E00E6
:103E80000E3A00005EBC62EF02F06170FF0E156E2C
:103E9000166E176E636A01EE10F0CC0EEE6EEE6ECB
:103EA000EE6EEE6EEE6EEE6EEE6EEE6EF00EEE6E90
:103EB000646A615077EC1FF0145077EC1FF03950B2
:103EC00077EC1FF0315077EC1FF0015077EC1FF0CA
:103ED000005077EC1FF0595077EC1FF0645077ECEE
:103EE0001FF0070E77EC1FF05E96AC8AFFD76426B2
:103EF000336E550E33B0010F33B2040F33B4100FCD
:103F000033B6400F326E550E33B8010F33BA040F7B
:103F100033BC100F33BE400F336E32C0EEFF33C0E0
:103F2000EEFF1200684369727473616D20737453FD
:103F3000726176202E3020346F4379706972686721
:103F400020742E446854726F6570322030302037F0
:103F500077772E776E7573756175656C656C7463B4
:103F60006F72696E7363632E2E6F6B75702F6F7235
:0E3F7000656A74632F7374737261702E7068CB
:020000040030CA
:0300010008121EC4
:020005008081F8
:060008000FC00FE00F40E5
:00000001FF
